:100000000C9454080C9474080C9474080C947408A0
:100010000C9474080C9474080C9474080C94740870
:100020000C9474080C9474080C9474080C94740860
:100030000C9474080C9474080C9474080C94740850
:100040000C9474080C9463130C9474080C94740846
:100050000C9474080C9474080C9474080C94740830
:100060000C9474080C94932B0C945F2B0C947408D0
:100070000C9474080C9485080C9474080C947408FF
:100080000C9474080C9474080C9474080C94740800
:100090000C9474080C9474080C9474080C947408F0
:1000A0000C9474080C9474080C9474080C947408E0
:1000B0000C9474080C9474080C9474080C947408D0
:1000C0000C9474080C9474080C9474080A737720C8
:1000D000310A000A737720300A00414D433A206EFE
:1000E0006F77204D300A00414D433A206E6F7720E4
:1000F0004D310A00414D433A2068616E646C6520C1
:10010000636C6F7365640A00414D433A204D3120A2
:1001100068616E646C652073746174757320636FBD
:100120007272656374696F6E0A00414D433A206EC6
:100130006F77204D320A00414D433A2068616E646A
:100140006C65206F70656E65640A00414D433A200E
:100150006E6F77204D330A00414D433A2068616E3F
:10016000646C65206F70656E65640A00414D433AAA
:10017000206E6F77204D340A00414D433A2068616C
:100180006E646C65206F70656E65640A00414D4356
:100190003A204D342068616E646C6520737461741C
:1001A000757320636F7272656374696F6E0A0041C4
:1001B0004D433A206E6F77204D350A00414D433A4A
:1001C0002068616E646C6520636C6F7365640A00FF
:1001D000414D433A206E6F77204D360A000A414D5B
:1001E00043206873776170206F75743A20000A535A
:1001F0004953383330304C0A004275696C742077AB
:10020000697468204156522D4743433A2000342EEA
:10021000362E320020616E64204156522D4C4942E8
:10022000433A2000312E382E30002072656C656113
:1002300073653A20003230313131323238000A6F82
:100240006E20004F6374203136203230313400206C
:100250002F200030373A30363A3533000A0A004151
:100260004D43207374617475733A204D000A005237
:10027000544D207374617475733A204D000A0A005E
:1002800020436F6D6D616E646C6973743A0A20531C
:10029000544154202D204669726D77617265205259
:1002A00065766973696F6E2C205374617475732C55
:1002B000206574632E2E2E0A2048454C50202D2098
:1002C0007468697320706167650A002072746D201C
:1002D0007A6F6E65333A200020616D63207A6F6E0D
:1002E00065333A20002072746D206D617463683A42
:1002F00020002072746D20636C6F7365640A0020A7
:1003000072746D206F70656E65640A002072746D82
:10031000206F70656E65640A002072746D206F70C6
:10032000656E65640A002072746D206F70656E657D
:10033000643A2000505752202B3132563A20002088
:100340006D560A4420202B332E33563A20200020AD
:100350006D560A4420202B322E35563A202000209C
:100360006D560A4420202B312E35563A202000208D
:100370004572617375726520454550524F4D202E70
:100380002E2E200020577269746520414435333386
:10039000383A2000205265616420414435333338B7
:1003A0000069326320627573206572726F720A0091
:1003B000756E6B6E6F776E20693263207374617433
:1003C000652000657272207374613A200065727254
:1003D00020736C613A2000657272206474613A2067
:1003E000000A0A534953383330304C206465627533
:1003F000672070726F6D70740A000A00574454438E
:1004000053523A20000A004D4D432046573A2000EF
:100410000A4275696C742077697468204156522DC0
:100420004743433A2000342E362E320020616E645A
:10043000204156522D4C4942433A2000312E382E4D
:1004400030002072656C656173653A20003230318E
:100450003131323238000A6F6E20004F6374203120
:1004600036203230313400202F200030373A3036F9
:100470003A3536000A004D435553523A20000A00DF
:100480007265737461727420616674657220636F43
:100490006C642072657365740A004D4F4453544177
:1004A00054455F504F5745524544202D3E204D4FF7
:1004B0004453544154455F574149545F5245534555
:1004C0005420000D0A004D4F4453544154455F578A
:1004D0004149545F5245534554202D3E204D4F44D1
:1004E00053544154455F574149545F465047415F1B
:1004F000444F4E4520000D0A004D4F445354415483
:10050000455F574149545F465047415F444F4E4510
:10051000202D3E204D4F4453544154455F46504793
:10052000415F52445920000D0A004D4F445354413D
:1005300054455F465047415F52445920000D0A0020
:10054000708A728E9290748C76989C9AA0A4889EE1
:10055000868478947A9682807C7EA207005101314D
:10056000000006C10003540201FF7F00703F00003D
:10057000040000620200040CC0077FEFABFF00C163
:10058000B7AD8A8F940202000000C6442B312E358D
:10059000560000000000000000000006005101317C
:1005A000000005C10003540201FF7F00703F0000FE
:1005B0000400007A0200040CC0077FEFABFF00F7D5
:1005C000F2E9A2A7AB0202000000C6442B322E358E
:1005D0005600000000000000000000020051013041
:1005E000000001C10003540101FF7F00703F008043
:1005F000010000010600040C00001946007DC955E9
:10060000504600050A0505000000C57446504741E4
:100610000000000000000000000000000051111662
:100620000001002B000000C00000CB5349533833B9
:1006300030304C52544D00005112130000002B007A
:100640000000C10000C8534953383330304C020019
:1006500051012F000008C00003540101FF7F00700A
:100660003F0080010000010600040C000019460054
:100670007DC955463C00050A0505000000C47452BA
:10068000544D0000000000000000000000000100C8
:10069000510135000007C0000340F26F0700000061
:1006A0000700000000000000000000000000000043
:1006B00000000000000000000000000000CA486FB9
:1006C000745377617052544D000000000000050023
:1006D000510131000004C10003540201FF7F00708A
:1006E0003F0000040000A10200040CC0077FEFAB34
:1006F000FF00F7F2E9A2A7AB0202000000C6442BFC
:10070000332E3356000000000000000000000400FB
:10071000510132000003C10003540201FF7F007049
:100720003F0000040000360200040CD0077FEFAB4E
:10073000FF00F7F2E9A2A7AB0202000000C7505782
:10074000522B313256000000000000000000030070
:10075000510131000002C10003540101FF7FFF7FFE
:100760003F0080010000010600040C0000193C322B
:1007700078E755463C00050A0505000000C67450A0
:100780006F776572000000000000000000000100AB
:10079000510132000000C1000340F26F0700000069
:1007A0000700000000000000000000000000000042
:1007B00000000000000000000000000000C7486FBB
:1007C0007453776170000000000000000000707238
:1007D0006F633A204E4554464E5F4150503A204395
:1007E0004D445F4745545F4445564943455F49443E
:1007F0000A0070726F633A204E4554464E5F53456F
:100800004E535F4556454E543A20434D445F534541
:10081000545F4556454E545F5245434549564552EF
:100820000A0070726F633A204E4554464E5F53453E
:100830004E535F4556454E543A20434D445F47451D
:10084000545F4556454E545F5245434549564552BF
:100850000A0070726F633A204E4554464E5F53450E
:100860004E535F4556454E543A20434D445F504CDD
:100870004154464F524D5F4556454E540A007072E2
:100880006F633A204E4554464E5F53454E535F4585
:1008900056454E543A20434D445F4745545F4445C6
:1008A000564943455F5344525F494E464F0A0070D4
:1008B000726F633A204E4554464E5F53454E535F28
:1008C0004556454E543A20434D445F4745545F4496
:1008D00045564943455F5344520A0070726F633A6C
:1008E000204E4554464E5F53454E535F4556454E48
:1008F000543A20434D445F5245535F444556494363
:10090000455F5344525F5245500A0070726F633A1C
:10091000204E4554464E5F53454E535F4556454E17
:10092000543A20434D445F4745545F53454E534F1F
:10093000525F52454144494E470A0070726F633A14
:10094000204E4554464E5F53454E535F4556454EE7
:10095000543A20434D445F4745545F53454E534FEF
:10096000525F5448524553484F4C44530A007072EA
:100970006F633A204E4554464E5F53454E535F4594
:1009800056454E543A20756E6B6E6F776E3A200066
:1009900070726F633A204E4554464E5F53544F5227
:1009A0004147453A20434D445F4745545F465255C1
:1009B0005F494E565F415245415F494E464F0A00DE
:1009C00070726F633A204E4554464E5F53544F52F7
:1009D0004147453A20434D445F524541445F4652AA
:1009E000555F444154413A2000414D430A0052545E
:1009F0004D0A0070726F633A204E4554464E5F5365
:100A0000544F524147453A20434D445F5752495451
:100A1000455F4652555F444154413A2000414D43A1
:100A20000A0052544D200070726F633A204E4554B4
:100A3000464E5F5049434D473A20434D445F47453A
:100A4000545F5049434D475F50524F50530A007016
:100A5000726F633A204E4554464E5F5049434D47AE
:100A60003A20434D445F4652555F434F4E54524FD8
:100A70004C3A2000414D430A0052544D0A00707216
:100A80006F633A204E4554464E5F5049434D473AB6
:100A900020434D445F4745545F4652555F4C4544A3
:100AA0005F50524F50530A0070726F633A204E45A8
:100AB00054464E5F5049434D473A20434D445F47AB
:100AC00045545F4C45445F434F4C4F525F43415048
:100AD00041420A0070726F633A204E4554464E5FA1
:100AE0005049434D473A20434D445F5345545F4678
:100AF00052555F4C45445F53544154450A0070724F
:100B00006F633A204E4554464E5F5049434D473A35
:100B100020434D445F4745545F4652555F4C454422
:100B20005F53544154450A0070726F633A204E453A
:100B300054464E5F5049434D473A20434D445F472A
:100B400045545F4652555F4C45445F5354415445AC
:100B5000206572723A000A0070726F633A204E4547
:100B600054464E5F5049434D473A20434D445F47FA
:100B700045545F4445565F4C4F4341545F52454393
:100B80005F49440A0070726F633A204E4554464EE6
:100B90005F5049434D473A20434D445F4652555FAD
:100BA000434F4E54524F4C5F43415041420A0070F4
:100BB000726F633A204E4554464E5F5049434D474D
:100BC0003A20434D445F5345545F414D435F504F7E
:100BD00052545F53544154450A0070726F633A2077
:100BE0004E4554464E5F5049434D473A20434D448D
:100BF0005F4745545F414D435F504F52545F5354DC
:100C00004154450A0070726F633A204E4554464E77
:100C10005F5049434D473A20434D445F4745545F39
:100C2000434C4F434B5F53544154450A0070726F1D
:100C3000633A204E4554464E5F5049434D473A2053
:100C4000434D445F5345545F4652555F41435449B9
:100C5000564154494F4E0A0070726F633A204E4518
:100C600054464E5F5049434D473A20434D445F53ED
:100C700045545F504F5745525F4C4556454C0A000E
:100C800070726F633A204E4554464E5F5049434D53
:100C9000473A20756E6B6E6F776E0A0070726F63E5
:100CA0003A204E4554464E5F56454E444F523A20E8
:100CB000434D445F524541445F52544D5F45450AA0
:100CC0000070726F633A204E4554464E5F56454E53
:100CD000444F523A20434D445F57524954455F5266
:100CE000544D5F45450A0070726F633A204E45547B
:100CF000464E5F56454E444F523A20434D445F4D59
:100D00004F444946595F52544D5F45455F57500A1D
:100D10000070726F633A204E4554464E5F56454E02
:100D2000444F523A20434D445F52455345545F4629
:100D30005047410A0070726F633A204E4554464E48
:100D40005F56454E444F523A20434D445F47455409
:100D50005F4649524D575F56455253494F4E0A0020
:100D600070726F633A204E4554464E5F56454E446E
:100D70004F523A20434D445F4745545F75445743B3
:100D80005F4441435F56414C55450A0070726F63A2
:100D90003A204E4554464E5F56454E444F523A20F7
:100DA000434D445F5345545F754457435F4441434B
:100DB0005F56414C55450A0070726F633A204E45AC
:100DC00054464E5F56454E444F523A20434D445F81
:100DD000524541445F52544D5F54454D505F56411A
:100DE0004C55450A0070726F633A204E4554464E8A
:100DF0005F56454E444F523A20434D445F5345544D
:100E00005F52544D5F54454D505F504F494E0A005C
:100E100070726F633A204E4554464E5F56454E44BD
:100E20004F523A20464F4F200A0052544D3A206EFE
:100E30006F77204D300A0052544D204D61736B3A4C
:100E4000200052544D3A204552524F523A204932D6
:100E500043206275732053444120737475636B2083
:100E60006C6F770A0052544D3A20636F6D70617455
:100E70006962696C69747920636865636B3A200004
:100E80006D730A0052544D3A206E6F77204D310A2F
:100E900000636F6D702E20636865636B3A20737515
:100EA00063636573730A00636F6D702E20636865FA
:100EB000636B3A206E6F206D6174636865732066A2
:100EC0006F756E640A0052544D204D61736B3A2069
:100ED000000A0052544D3A2068616E646C652063CC
:100EE0006C6F7365642C20656467650A0052544D0D
:100EF0003A2068616E646C6520636C6F7365642C66
:100F0000204D30206C6576656C0A0052544D3A20B5
:100F10006D6F64756C652072656D6F7665640A002F
:100F200052544D3A206E6F77204D320A0052544D84
:100F3000204D61736B3A200052544D3A2068616E27
:100F4000646C65206F70656E65640A0052544D3A9A
:100F5000206D6F64756C652072656D6F7665640ACF
:100F60000052544D3A206E6F77204D330A00525490
:100F70004D3A206E6F77204D340A0052544D204D6B
:100F800061736B3A200052544D3A2053657475706A
:100F9000204457435F44414320746F203256350A42
:100FA0000052544D3A2068616E646C65206F706524
:100FB0006E65640A0052544D3A206D6F64756C651D
:100FC0002072656D6F7665640A0052544D3A205365
:100FD0006574646F776E204457435F4441430A0051
:100FE00052544D3A206E6F77204D350A0052544DC1
:100FF000204D61736B3A200052544D3A2053657472
:10100000646F776E204457435F4441430A00525453
:101010004D3A206D6F64756C652072656D6F7665F5
:10102000640A0052544D3A206E6F77204D360A0004
:1010300052544D204D61736B3A200052544D3A206A
:101040006D6F64756C652072656D6F7665640A00FE
:101050000A616D6320776974686F7574207A332034
:101060007265636F7264730A000A72746D20776927
:1010700074686F7574207A33207265636F7264735D
:101080000A000A666F7220616D633A2000666F7213
:101090002072746D3A20000A52544D2068737761B3
:1010A00070206F75743A200011241FBECFEFD1E27B
:1010B000DEBFCDBF13E0A0E0B2E0E8E1FFE500E075
:1010C0000BBF02C007900D92A23DB107D9F71BBE1E
:1010D0001AE0A2EDB3E001C01D92A036B107E1F71E
:1010E0000E947B2C0C948A2F0C9400001092100408
:1010F00010927C0087EC80937A0080917A0084FFC4
:10110000FCCF8FEC80937A0008951F920F920FB658
:101110000F920BB60F9211242F934F935F936F93FF
:101120007F938F939F93AF93BF93EF93FF938091A0
:10113000780090917900A0E0B0E04091D203509106
:10114000D3036091D4037091D503840F951FA61F1C
:10115000B71F8093D2039093D303A093D403B0938B
:10116000D5032091D6032F5F2093D6032223E9F4E1
:1011700020911004E22FF0E0EE0FFF1FE85FFB4F1D
:10118000892F9A2FAB2FBB27918380831092D20394
:101190001092D3031092D4031092D503822F8F5F45
:1011A00083708093100480937C008FEC80937A008E
:1011B000FF91EF91BF91AF919F918F917F916F912F
:1011C0005F914F912F910F900BBE0F900FBE0F901C
:1011D0001F901895E82FF0E0E370F070EE0FFF1FFE
:1011E000E85FFB4F8081918108951F93CF93DF9338
:1011F000CDB7DEB7C354D0400FB6F894DEBF0FBEF4
:10120000CDBF182F8DED91E00E94CD2B812F0E9434
:10121000462C80E092E00E94BB2B809139098C83A0
:1012200080E18D838091EE088F83809138098887D3
:101230008C5F8093380982E0898784E08A8782EF17
:101240008B871C868FE68D871E878BE08B83CE0174
:1012500001960E941B1481E08A83CE0101960E94B0
:10126000DD1010930202CD5BDF4F0FB6F894DEBFA6
:101270000FBECDBFDF91CF911F910895CF9380E82E
:101280000E94CC2AC82F809104028093030280918F
:10129000DD03809304028091DE03C81749F0CC235C
:1012A00019F08CEC90E002C083ED90E00E94CD2B11
:1012B00080E80E94CC2A9091DC03882319F09D7F5E
:1012C000916002C092609E7F9093DC038091040243
:1012D000833009F482C0843040F49091030281305D
:1012E00071F1823008F058C00AC0853009F4D3C0CB
:1012F000853008F498C0863009F00DC1F0C09923FC
:1013000009F406C18AED90E00E94CD2B80E060E0F8
:1013100041E050E00E941B1181E060E041E050E0BC
:101320000E941B1182E060E043E050E00E941B112C
:1013300082E060E040E050E00E941B11E9C0913083
:1013400051F080E060E041E050E00E941B1187EE28
:1013500090E00E94CD2B8091DE03C81771F0CC2362
:1013600061F0C093DE0384EF90E00E94CD2B80E01B
:101370000E94F50882E08093DD038091DE03C817A8
:1013800009F445C0CC2309F042C01092DE0388E086
:1013900091E00E94CD2B3BC0923021F08AE291E097
:1013A0000E94CD2B8091DE03C81771F0CC2361F42D
:1013B0001092DE0387E391E00E94CD2B81E00E9432
:1013C000F50881E08093DD038091DB03882309F435
:1013D000A2C01092DB0383E09CC0809103028330A3
:1013E00021F08BE491E00E94CD2B8091DE03C817A1
:1013F00071F0CC2361F41092DE0388E591E00E9445
:10140000CD2B81E00E94F50881E08093DD0380917F
:10141000DA03882309F47FC01092DA0381E0809315
:10142000ED0884E076C080910302843021F08CE6E0
:1014300091E00E94CD2B8091DE03C81781F0CC2370
:1014400071F41092DE0389E791E00E94CD2B81E0D8
:101450000E94F50885E08093DD031092E5088091F5
:10146000DE03C81741F0CC2331F0C093DE038DE8D2
:1014700091E00E94CD2B8091D803882309F44BC0C2
:101480001092D80387E08093ED0886E08093DD0317
:101490001092E50840C080910302853021F08FEA68
:1014A00091E00E94CD2B8091DE03C81771F0CC2310
:1014B00061F0C093DE038CEB91E00E94CD2B80E0C5
:1014C0000E94F50884E08093DD038091D90388238E
:1014D00079F01092D90386E08093DD0309C08091F2
:1014E0000302863029F00D9A80ED91E00E94CD2B09
:1014F0008091D803882329F01092D80387E0809345
:10150000ED088091ED08882331F482E00E94F5080F
:1015100081E08093DD038091D703882329F18091B6
:10152000DC0380FF03C080E00E94F5088091DC03AB
:1015300081FF03C081E00E94F5088091DC0382FFF7
:1015400003C082E00E94F5088091DC0383FF03C0A2
:1015500083E00E94F5088091DC0384FF03C084E0EF
:101560000E94F5081092D703CF910895809104024C
:1015700008958091DC03089581E08093DB03089552
:1015800081E08093DA031092D9031092D803089572
:1015900081E08093D9031092DA031092D803089562
:1015A00081E08093D8031092D9031092DA03089552
:1015B00081E08093D70308956F927F928F929F92DC
:1015C000AF92BF92CF92DF92EF92FF920F931F9351
:1015D000CF93DF93CDB7DEB7C850D1400FB6F894A4
:1015E000DEBF0FBECDBF4C01E62E3A01FC011082DA
:1015F000CE01019660E070E048E050E00E945A2F72
:10160000FE01319697E080E02191820F9150E1F741
:1016100081959885891709F059C00E8110E093E0F3
:10162000000F111F9A95E1F70115110509F450C03B
:1016300089E0A82EB12CAC0EBD1EB80160507040E0
:10164000CE01019645E050E00E945A2F8A8199818F
:10165000890FFB808F0D9C81890F81959D81891752
:10166000C9F5CF2CDD240B5F1F4FB80160507040CF
:10167000C501A6010E945A2F20E030E006C08A0D65
:101680009B1DFC018081280F3F5F832F90E08C150C
:101690009D05A8F321958C812817F1F48C85803362
:1016A00079F4F40180818F5F80838E1549F4611491
:1016B000710431F0C301B5014F2D50E00E94512F4C
:1016C0008A8187FD0BC00C0D1D1DB7CF82E007C0BE
:1016D00083E005C084E003C085E001C080E0C85F0E
:1016E000DE4F0FB6F894DEBF0FBECDBFDF91CF91B6
:1016F0001F910F91FF90EF90DF90CF90BF90AF9030
:101700009F908F907F906F900895EF92FF920F932C
:101710001F93CF93DF93CDB7DEB728970FB6F8941A
:10172000DEBF0FBECDBF7C01CE01019660E070E050
:1017300048E050E00E945A2FFE01319697E080E089
:101740002191820F9150E1F781959885891749F58C
:101750000E8110E023E0000F111F2A95E1F701151B
:10176000110509F1B80160507040CE01019645E0C5
:1017700050E00E945A2F2A819981920F8B81980FF5
:101780003C81930F91953D81931779F490E00596F4
:10179000080F191F27FFE6CFF7011183008380E0B0
:1017A00005C082E003C083E001C084E028960FB644
:1017B000F894DEBF0FBECDBFDF91CF911F910F9187
:1017C000FF90EF90089589E193E00E94CD2B80E097
:1017D000089580E892E00E94CD2B80E00895CF9399
:1017E000DF9300D0CDB7DEB784E993E00E94CD2B24
:1017F0008CE061E0AE014F5F5F4F0E94AE2888230E
:1018000029F085E092E00E94BB2B0AC08DE092E0B7
:101810000E94BB2B89810E94462C8A810E94462C03
:1018200082E192E00E94BB2B80E00F900F90DF914D
:10183000CF910895CF93DF9300D000D0CDB7DEB71E
:1018400019821A821B821C828CE289838CE18A8332
:10185000A7E4B4E0FE01319680E090E03D91232FB3
:1018600020532A3008F027502193019684309105A7
:10187000A9F789818295807F9A819F70892B8983BE
:101880008B818295807F9C819F70892B8A8384E8DD
:1018900093E00E94CD2B89810E94462C8A810E9470
:1018A000462C8CE061E0AE014F5F5F4F0E948A25BD
:1018B000882319F084E192E002C080E292E00E9465
:1018C000BB2B80E00F900F900F900F90DF91CF9186
:1018D0000895CF93DF938FE693E00E94CD2BC0E075
:1018E000D0E080E5BE0140E00E949024219682E095
:1018F000C030D807B1F78BE292E00E94BB2B80E0AA
:10190000DF91CF910895EF92FF920F931F93CF93A2
:10191000DF9300D000D000D0CDB7DEB782E392E0F5
:101920000E94BB2B81E56AEF70E046E050E09E012B
:101930002F5F3F4F0E94ED24882329F084E492E03A
:101940000E94BB2B10C07E010894E11CF11C00E03A
:1019500010E0F70181917F010E94462C0F5F1F4F1D
:1019600006301105B1F782E192E00E94BB2B80E0C6
:1019700026960FB6F894DEBF0FBECDBFDF91CF9194
:101980001F910F91FF90EF900895CF93DF9380E028
:101990000E94EA08EC0184E393E00E94CD2BBE0193
:1019A00080E090E024E63DE84DE050E00E94E92E22
:1019B0000E94FD2B81E00E94EA08EC018FE393E096
:1019C0000E94CD2BBE0180E090E022E836E044E0AA
:1019D00050E00E94E92E0E94FD2B82E00E94EA085E
:1019E000EC018FE493E00E94CD2BBE0180E090E0FB
:1019F0002BEE37E040E050E00E94E92E0E94FD2BE4
:101A000083E00E94EA08EC018FE593E00E94CD2B71
:101A1000BE0180E090E020E13AE340E050E00E9427
:101A2000E92E0E94FD2B8EE492E00E94BB2B80E009
:101A3000DF91CF910895EF92FF920F931F93CF9371
:101A4000DF9300D0CDB7DEB786E293E00E94CD2BC6
:101A5000CE0101960E94922290E00E94FD2B03E5A8
:101A600012E0C8010E94BB2B89819A810E94FD2B44
:101A700022E1E22E22E0F22EC7010E94BB2BCE0112
:101A800001960E94850B90E00E94FD2BC8010E94E8
:101A9000BB2B89819A810E94FD2BC7010E94BB2B21
:101AA00080E00F900F90DF91CF911F910F91FF90E9
:101AB000EF9008958CE093E00E94CD2B86E00E9489
:101AC000292080E008958FEF92E00E94CD2B81E0E5
:101AD0000E94292080E0089582EF92E00E94CD2BA1
:101AE00080E00E94292080E0089585EE92E00E9427
:101AF000CD2B0E94AB2390E00E94FD2B82E192E06F
:101B00000E94BB2B88E00E94292080E00895CF939B
:101B1000DF930F92CDB7DEB788ED92E00E94CD2B18
:101B2000CE01019660E040E050E00E94DC0A90E0C7
:101B30000E94FD2B83E592E00E94BB2B898190E0FF
:101B40000E94FD2B82E192E00E94BB2B87E00E9465
:101B5000292080E00F90DF91CF910895CF93DF93FC
:101B60000F92CDB7DEB78BEC92E00E94CD2BCE0169
:101B7000019660E040E050E00E94002390E00E9467
:101B8000FD2B83E592E00E94BB2B898190E00E94AF
:101B9000FD2B82E192E00E94BB2B85E00E94292070
:101BA00080E00F90DF91CF9108958EEE91E00E943A
:101BB000CD2B89EF91E00E94CD2B8EE092E00E9428
:101BC000CD2B84E192E00E94CD2B84E292E00E9432
:101BD000CD2B8AE292E00E94CD2B85E392E00E9419
:101BE000CD2B8EE392E00E94CD2B83E492E00E9405
:101BF000CD2B8FE492E00E94CD2B83E592E00E94F2
:101C0000CD2B8CE592E00E94CD2B8FE592E00E94D7
:101C1000CD2B0E94B60A90E00E94FD2B8DE692E04B
:101C20000E94CD2B8FE692E00E94CD2B0E941120C6
:101C300090E00E94FD2B8DE792E00E94CD2B80E08A
:101C4000089585E592E00E94BB2B1092410408950F
:101C5000CF93DF93AC01A0E08A2F90E0880F991F0B
:101C6000880F991FFC01EF53FD4F60817181B0E037
:101C70002B2F30E0FB01E20FF31FE081EE2359F040
:101C8000240F351FE90128812E272F7511F4BF5F1E
:101C9000EFCFAF5FE1CFBB2349F08F539D4FDC0106
:101CA0001296ED91FC911397099501C081E0DF91A7
:101CB000CF910895CF93DF930F92CDB7DEB7CE01CA
:101CC00001960E94412B882309F04CC089818830FD
:101CD00019F08D3081F510C080914104882309F4FA
:101CE00041C081508093410488E00E94222B80E211
:101CF0000E94222B88E034C08AE00E94222B8DE0D3
:101D00000E94222BE0914104EE2371F0F0E0EE5BA3
:101D1000FB4F108282E494E00E94280E882321F079
:101D20008FE592E00E94BB2B1092410480E792E085
:101D30000E94BB2B17C08B31A9F0909141049032C7
:101D400070F40E94222B80914104E82FF0E0EE5BBA
:101D5000FB4F998190838F5F8093410403C087E09C
:101D60000E94222B0F90DF91CF9108950F931F9324
:101D7000CF93DF93C7E3D0E0CE010E946A2F90E0BB
:101D80008F70907024E630E0829F8001839F100D59
:101D9000929F100D1124CE0101960E946A2F90E0AF
:101DA0008F7090709C01220F331F53E0880F991F92
:101DB0005A95E1F7280F391F020F131FCE01029623
:101DC0000E946A2F8F709801280F311DC901DF9181
:101DD000CF911F910F910895CF92DF92EF92FF92D2
:101DE0000F931F9387E390E00E946A2F90E08F701B
:101DF000907024E630E0829F6001839FD00C929F18
:101E0000D00C1124EE24D7FCE094FE2C88E390E063
:101E10000E946A2F90E08F7090709C01220F331FF8
:101E200063E0880F991F6A95E1F7280F391FC901F0
:101E3000AA2797FDA095BA2FC80ED91EEA1EFB1E31
:101E400089E390E00E946A2F8F70A7019601280F06
:101E5000311D411D511DDA01C901529AEFE9FFE020
:101E60003197F1F700C000005298E0E2F0E000E0A6
:101E700010E020E030E8539AB901A8014823592323
:101E80006A237B23411551056105710509F05398BB
:101E9000F894529A52987894369527951795079505
:101EA000319749F71F910F91FF90EF90DF90CF90FE
:101EB000089590E29093B8008E7F8093BA001092BC
:101EC000BD0084E48093BC0010926C0410926B04FB
:101ED0000895CF938091BC0087FF67C0C091B9007F
:101EE000C87FC03661F0C13620F4CC2309F448C065
:101EF00051C0C038D1F0C03A09F04CC02BC010928C
:101F0000E103E091F308F091F40880818068808318
:101F100080818E7F80838091BB00838381E080936A
:101F2000E10394EC9093BC0012C0E091F308F091AF
:101F3000F4088091E1039091BB00E80FF11D9383B9
:101F40008F5F8093E10384EC8093BC0081E08093F9
:101F5000E0032BC0E091F308F091F4088091E103D5
:101F6000828380818160808380818F77808384EC0D
:101F70008093BC001092E0038AE080931C0315C09C
:101F800081EA93E00E94CD2B8091BC008069809310
:101F9000BC000BC080EB93E00E94CD2B8C2F0E94E5
:101FA000462C81E093E00E94BB2B8091E003CF910F
:101FB0000895CF92DF92FF920F931F93CF93DF93F9
:101FC0000F92CDB7DEB78091DF03882341F4909163
:101FD0006C0480916B04981709F053C0E5C08F3FE3
:101FE00039F484E60E94ED2A8EEF8093DF03DCC093
:101FF0008E3F09F046C080919D08882311F14091E1
:102000006B0450E023E430E0429FC001439F900DF9
:10201000529F900D112483599B4F0E94D91F90917C
:102020006A04891771F480916B048F5F80936B044D
:10203000803111F410926B041092DF0310929D080E
:10204000B3C00E94FD2A882309F4AEC08091E20348
:1020500081508093E203882321F084E60E94ED2AD8
:1020600010C080916B048F5F80936B04803111F4FA
:1020700010926B0483E093E00E94BB2B1092DF036D
:1020800093C084EA8093BC008091BC0087FFFCCFA2
:102090001091B900187F183059F083EC93E00E943A
:1020A000CD2B812F0E94462C81E093E00E94BB2B18
:1020B00020916B0430E083E490E0289FF001299F99
:1020C000F00D389FF00D1124E359FB4F838180936D
:1020D000BB0084E88093BC008091BC0087FFFCCFEC
:1020E0001091B900187F183159F08DEC93E00E94DF
:1020F000CD2B812F0E94462C81E093E00E94BB2BC8
:1021000011E083E4C82ED12C94E8F92E04E923C011
:10211000181719F40093BC001DC0E10FF11D838155
:102120008093BB00F092BC008091BC0087FFFCCF85
:102130002091B900287F283269F087ED93E0298348
:102140000E94CD2B2981822F0E94462C81E093E0B2
:102150000E94BB2B1F5F20916B04822F90E08C9D0F
:10216000F0018D9DF00D9C9DF00D1124E359FB4F66
:102170008281811768F68181813059F48091DF0373
:102180008E3F79F08FEF8093DF0383E08093E2034B
:1021900008C0822F8F5F80936B04803111F41092FE
:1021A0006B0484EC8093BC000F90DF91CF911F9162
:1021B0000F91FF90DF90CF90089560916C04462FAF
:1021C00050E023E430E0429FF001439FF00D529F26
:1021D000F00D1124E359FB4FDC0183E40D900192D3
:1021E0008150E1F76F5F60936C04603111F41092DD
:1021F0006C0480E0089591E090939D0880936A04B8
:102200000895DA01A90190E026E130E0829FF00113
:10221000839FF00D929FF00D1124E256F74F6187D6
:1022200010861286B183A083128213825583448361
:1022300016821782089590E026E130E0829FD00157
:10224000839FB00D929FB00D1124A256B74F662305
:10225000D1F412968C91129790E0880F991FED910E
:10226000FC911197E80FF91F5183408312968C91CE
:1022700012978F5F12968C9312978430F1F4129616
:102280001C921297089516968C91169790E0880FDD
:10229000991F1496ED91FC911597E80FF91F518342
:1022A000408316968C9116978F5F16968C9316978F
:1022B000843019F416961C9216970895CF93DF93E5
:1022C000EA0190E026E130E0829FD001839FB00DCB
:1022D000929FB00D1124A256B74F662309F51396AD
:1022E0008C91139712969C9112978917D9F190E0CF
:1022F000880F991FED91FC911197E80FF91F8081CC
:1023000091819983888313968C9113978F5F13968D
:102310008C931397843041F513961C92139724C025
:1023200017968C91179716969C9116978917D1F04E
:1023300090E0880F991F1496ED91FC911597E80F86
:10234000F91F808191819983888317968C911797C3
:102350008F5F17968C931797843031F417961C92E1
:10236000179702C081E001C080E0DF91CF9108950E
:10237000EF92FF920F931F93CF93DF9300D0CDB7CF
:10238000DEB7F82E282F30E086E190E0289F80010C
:10239000299F100D389F100D11240256174FF80178
:1023A0008085882309F0BCC08285813041F081306E
:1023B00068F0823089F0833009F04BC028C025B125
:1023C000F80191859095922395B942C085B1F801A5
:1023D0009185892B85B93BC0F8018585882349F013
:1023E00095B181858095892385B9858581508587BB
:1023F0000BC0F8018685882339F085B19185892B3A
:1024000085B9868581508687F80186851AC0F801CE
:102410008685882341F085B19185892B85B986858C
:10242000815086870CC0F8018585882341F095B1DD
:1024300081858095892385B9858581508587F801B7
:102440008585882331F4838585878485868781E027
:102450008787F801E784F1E0EF1609F0CEC08F2DF1
:1024600061E0AE014F5F5F4F0E945E11882321F54E
:10247000F801E08649815A81CA019070009711F4F1
:10248000108A4BC09C01215030402A3F310540F456
:1024900082E0F801808B518B428B538B448B3DC083
:1024A0008C3F910519F4F801108637C08F3F9105D4
:1024B000A1F5F801E08A31C08F2D60E0AE014F5FD9
:1024C0005F4F0E945E11882341F589819A81907047
:1024D0008130910551F08130910550F082309105A5
:1024E00051F083309105C9F40FC0F801E28615C0A0
:1024F000F801128612C09AE0F80193878AE5848772
:102500009587868782E008C09AE5F80193878AE07C
:1025100084879587868783E08287F80117866DC058
:10252000F8018089813039F0813060F0823081F0AB
:10253000833081F519C025B1F801918590959223DA
:1025400095B927C085B1F8019185892B85B920C03F
:10255000F8018489882341F085B19185892B85B95B
:1025600084898150848B0CC0F8018389882341F0D1
:1025700095B181858095892385B983898150838B25
:10258000F8018389882331F48189838B8289848B44
:1025900081E0858BF8018589882379F18F2D61E0B1
:1025A000AE014F5F5F4F0E945E11882321F561E00D
:1025B000F801608749815A81CA019070009711F42F
:1025C000108A19C09C01215030402A3F310540F447
:1025D00082E0F801808B518B428B538B448B0BC074
:1025E0008C3F910519F4F801108605C08F3F9105C5
:1025F00011F4F801608BF801158A0F900F90DF91AC
:10260000CF911F910F91FF90EF900895DB0190E023
:1026100026E130E0829FF001839FF00D929FF00D44
:102620001124E256F74F80858C93828511968C9306
:102630001197848512968C931297838513968C93A9
:102640001397808914968C931497828915968C938E
:102650001597818916968C9316970895CF92DF92DD
:10266000EF92FF920F931F93CF93DF930F92CDB70B
:10267000DEB77B0189830E94042A898181600E94E0
:10268000272A882321F40E941C2A81E012C081E0BD
:102690000E945C2A182F00E080E00E945C2AC82E6D
:1026A000DD24C02AD12A0E941C2AF701D182C082CF
:1026B00080E00F90DF91CF911F910F91FF90EF90ED
:1026C000DF90CF9008951F920F920FB60F920BB626
:1026D0000F9211242F933F934F935F936F937F93A8
:1026E0008F939F93AF93BF93EF93FF930E948C2A96
:1026F0008091E3039091E403A091E503B091E60398
:102700000196A11DB11D8093E3039093E403A09370
:10271000E503B093E6038091E7039091E803019607
:102720009093E8038093E70323E0883E920739F40F
:1027300081E08093E3081092E8031092E703809110
:10274000E9038F5F8093E903843629F481E0809365
:10275000E4081092E9038091EA038F5F8093EA0313
:102760008A3071F40E94032B81E08093F00810926C
:10277000EA0380910504882319F0815080930504B1
:10278000FF91EF91BF91AF919F918F917F916F9149
:102790005F914F913F912F910F900BBE0F900FBE05
:1027A0000F901F90189585B1817F85B9209A289840
:1027B0008FEC97E00197F1F700C0000021E0199B32
:1027C00020E081E01A9B80E091E01B9B90E0289A3A
:1027D000EFECF7E03197F1F700C0000063B141E0A2
:1027E0001A9B40E031E01B9B30E051E061FF50E07C
:1027F000251322E0841382E0931392E0E82FEE0F7A
:10280000E80FE20F89E0989F902D1124E90FF0E086
:10281000E05CFA4F8491089590E08057904062E028
:1028200070E00E94142F862F0895FC018481869504
:10283000869581700895FC0183819481890F81952B
:1028400085838281DF0123E090E005C015963C91ED
:102850001597930F2F5F11962817C0F3DF01A80F6C
:10286000B11D919513969C9313978F5F8283089562
:10287000CF93DF93EC0188818E7F806888830E94EC
:10288000D90F88818F77888380E0DF91CF91089579
:10289000FC0183819481890F819595819817D9F4E2
:1028A000828190E0019753E040E008C02E0F3F1F67
:1028B000D90113962C911397420F5F5F252F30E0BB
:1028C000281739079CF3E80FF91F41958381841776
:1028D00021F082E0089581E0089580E008959F92BC
:1028E000AF92BF92CF92DF92EF92FF920F931F931E
:1028F000CF93DF93CDB7DEB760970FB6F894DEBF06
:102900000FBECDBF8C017B01FE013296AEE5B3E078
:1029100086E00D9001928150E1F7D80114962C9138
:102920001497269526952A3009F447C32B3040F496
:10293000243009F44FC0263011F00C94951F09C0C3
:102940002C3209F48FC4203311F00C94951F0C9491
:102950002A1DF8018085813011F00C94951F8EECB2
:1029600097E00E94CD2BD80116968C911697F7010F
:10297000838317969C91179714968C9114978C5F6C
:102980008C7F292F2370822B84838091EE0886838D
:1029900014968C91149783709C7F892B878318964B
:1029A0008C91189780871186128681E8838782E050
:1029B000848783E7858781E586878BE287878DEB30
:1029C000808B82E9818B128A138A83E8848B82E16F
:1029D0000C94D41FD80118968C911897803209F462
:1029E0009FC0813248F4813009F446C0813088F0BC
:1029F000823009F0D9C26EC0823209F45EC18232DF
:102A000008F4BDC0873209F41AC28D3209F0CCC275
:102A100084C182EF97E00E94CD2BF80181858093DD
:102A20003909828580933A098681D70113968C9360
:102A30001397978184818C5F8C7F292F2370822B41
:102A400014968C9314978091EE0816968C93169793
:102A5000848183709C7F892B17968C931797808530
:102A600018968C93189719961C920E94D80A0E9467
:102A7000252087E00C94AE1E82E298E00E94CD2BC8
:102A8000D80116968C911697F701838317969C911F
:102A9000179714968C9114978C5F8C7F292F237035
:102AA000822B84838091EE08868314968C911497F0
:102AB00083709C7F892B878318968C9118978087C9
:102AC000118680913909828780913A09838789E04C
:102AD0000C94D41F82E598E00E94CD2BD801169665
:102AE0008C911697F701838317969C9117971496EC
:102AF0008C9114978C5F8C7F292F2370822B848379
:102B00008091EE08868314968C91149783709C7F35
:102B1000892B878318968C91189780871186FBC222
:102B20008EE798E00E94CD2BD80116968C911697CF
:102B3000F701838317969C91179714968C9114979D
:102B40008C5F8C7F292F2370822B84838091EE08E9
:102B5000868314968C91149783709C7F892B87832E
:102B600018968C91808711860E94EC29D7011A96BD
:102B70008C931A9781E01B968C931B97CCC08FEA9D
:102B800098E00E94CD2BF8018681D70113968C9393
:102B90001397978184818C5F8C7F292F2370822BE0
:102BA00014968C9314978091EE0816968C93169732
:102BB000848183709C7F892B17968C9317978085CF
:102BC00018968C93189719961C92A384BB2494850D
:102BD00080E0A82AB92AC58496840E94EC2901972E
:102BE000A816B90629F48FEFF7018287838708C0FA
:102BF000C5010196D7011A968C931A971B969C9340
:102C0000F501EE0FFF1FEC59FC4F0C2D10E0608119
:102C10007181600F711FC7010C96492D50E00E9411
:102C20003B2FB5E0BC1560F0C801890D911D8530C2
:102C3000910534F0F701E01BF10B8091EE08818BD8
:102C4000E2E0AE16B104C8F4FDE0FC1570F1DD243D
:102C5000C601890D911D8D3091053CF1F701EC19EC
:102C6000FD098091EE0890E08057904062E070E0AE
:102C70000E94142F605A618F18C049E04C15A8F0CB
:102C8000DD24C601890D911D8930910574F0F7018D
:102C9000EC19FD098091EE0890E08057904062E0C9
:102CA00070E00E94142F605A658B892D875FD701D1
:102CB00012968C9312970C94B81F8BED98E00E949B
:102CC000CD2BF8018681D70113968C9313979781AA
:102CD00084818C5F8C7F292F2370822B14968C9398
:102CE00014978091EE0816968C93169784818370C2
:102CF0009C7F892B17968C931797808518968C93B9
:102D0000189719961C92199781E01A968C931A9726
:102D10001B961C921B9789E0CBCF8BE099E00E9419
:102D2000CD2BF8018681D70113968C931397978149
:102D300084818C5F8C7F292F2370822B14968C9337
:102D400014978091EE0816968C9316978481837061
:102D50009C7F892B17968C931797808518968C9358
:102D6000189719961C92199781859AE012969C9350
:102D700012978430C9F1853058F4813009F18130DF
:102D800098F0823001F1833011F00C94B81F1EC00E
:102D9000863009F43FC08630D8F18730E9F18830B9
:102DA00011F00C94B81F48C0F701128680EC83879D
:102DB0000E94B90AD7011C968C931C970C94B81FDB
:102DC0008091E1080AC08091E70815C080E00E9468
:102DD000EA089695879596958795F701828780E40E
:102DE000838714860C94B81F81E00E94EA089695A8
:102DF000879596958795D7011A968C931A9780E4B4
:102E00001B968C931B971C961C921C970C94B81FB6
:102E100082E0DDCF83E0E9CFF701128680EC838783
:102E20000E941420D7011C968C930E941420F70155
:102E300095878BE00C94D41F8091F208DCCF8BE354
:102E400099E00E94CD2BF8018681D70113968C93CF
:102E50001397978184818C5F8C7F292F2370822B1D
:102E600014968C9314978091EE0816968C9316976F
:102E7000848183709C7F892B17968C93179780850C
:102E800018968C93189719961C92199781858430FF
:102E900009F43CC0853050F48130B9F0813090F0B5
:102EA0008230E9F0833009F07DC026C0863009F415
:102EB00041C08630A8F1873009F474C0883009F029
:102EC00071C042C0F7010C94D21F8FE3D7011A964C
:102ED0008C931A9780916A0390916B0309C08FE3DA
:102EE000D7011A968C931A9780916C0390916D0379
:102EF000FC01B996E49133C08FE3D7011A968C9305
:102F00001A9780916E0390916F03F2CF8FE3D701F0
:102F10001A968C931A978091700390917103E8CF61
:102F20008FE3D7011A968C931A9780917203909130
:102F30007303DECF8FE3D7011A968C931A97809193
:102F4000740390917503D4CF8FE3F701828780914A
:102F5000780390917903FC01B996E491D7011B960F
:102F6000EC931B97FC01B896E4911C96EC931C978C
:102F7000FC01B796E4911D96EC931D97FC01B69663
:102F8000E4911E96EC931E97FC01B596E4911F9672
:102F9000EC931F978496FC01849150968C935097E4
:102FA0008EE086CED7011EC48EE699E00E94CD2B1E
:102FB000F80180850E94462C48C5D80118968C914E
:102FC0001897813109F452C0823109F4B2C08031BE
:102FD00009F0ABC780E999E0288B0E94CD2BF8015E
:102FE00081852889882351F08130D1F4288B0E9473
:102FF00011202889882311F483ED13C0D7011A9674
:103000001C921A9782E01B968C931B971C961C921D
:103010001C9719961C92199712962C93129705C01B
:1030200089ECF701818787E08283D80116968C911D
:103030001697F701838317969C91179714968C9196
:1030400014978C5F8C7F292F2370822B848380912F
:10305000EE08868314968C91149783709C7F892B3D
:10306000878318968C911897808782C780EC99E0A7
:103070000E94CD2BD80116968C911697F701838369
:1030800017969C91179714968C9114978C5F8C7F50
:10309000292F2370822B84838091EE0886831496D7
:1030A0008C91149783709C7F892B878318968C91C1
:1030B0001897808711861A96AC901A97BB241B9696
:1030C0009C911B9780E0A82AB92A1C96CC901C974B
:1030D000C28619968C911997882321F0813009F0C6
:1030E00047C70EC089EE99E00E94CD2BB501605014
:1030F0007040C7010B964C2D50E00E945A2F16C00D
:103100008EEE99E00E94CD2B0E941120882329F495
:1031100083EDF701818787E047C79701255F3F4F20
:1031200080E5B5014C2D50E00E9435228C2D885F42
:10313000BECD83EF99E00E94CD2BF801C280F6EF5F
:10314000CF0ED8011A96AC901A97BB241B969C916F
:103150001B9780E0A82AB92A19968C911997882381
:1031600021F0813009F05DC014C08DE19AE00E9429
:10317000CD2BF701C286B50160507040C8010C9696
:103180004C2D50E00E94722FD70119961C9219976E
:1031900048C082E29AE00E94CD2B80E593E00E9435
:1031A000BB2BC5010E94FD2B86E593E00E94BB2B43
:1031B0008C2D90E00E94FD2B8EE493E00E94BB2BAF
:1031C0000E941120F701882349F1C28611868CE7FD
:1031D000BE016F5F7F4F0E949B208823B1F46981FD
:1031E00061616F7769838CE70E94C020882311F0AA
:1031F000F70114C09801245F3F4F80E5B5014C2DC5
:1032000050E00E94C524882361F0D7011A961C92D1
:103210001A9783ED19968C93199703C0128683ED44
:103220008187D80116968C911697F701838317969C
:103230009C91179714968C9114978C5F8C7F292FF3
:103240002370822B84838091EE08868314968C9160
:10325000149783709C7F892B878318968C9118977D
:103260008087A1C6D80118968C9118978C3009F4E4
:1032700068C38D30A8F4853009F4B7C0863030F4C7
:10328000882321F1843009F0C8C357C0873009F47E
:10329000E2C0873008F4DCC0883009F0BEC361C1E9
:1032A000893109F415C38A3138F48D3009F4C3C269
:1032B000813109F0B2C375C38E3109F406C38D3272
:1032C00009F43CC38A3109F0A8C335C387E29AE008
:1032D0000E94CD2BF8018681D70113968C9313970A
:1032E000978184818C5F8C7F292F2370822B149689
:1032F0008C9314978091EE0816968C931697848180
:1033000083709C7F892B17968C93179780851896CE
:103310008C93189719961C9219971A961C921A97C3
:1033200082E31B968C931B9781E01C968C931C97D1
:103330001D961C921D978BE0BBCC8FE49AE00E94F7
:10334000CD2BF8018681D70113968C931397978123
:1033500084818C5F8C7F292F2370822B14968C9311
:1033600014978091EE0816968C931697848183703B
:103370009C7F892B17968C931797808518968C9332
:10338000189719961C9219971A961C921A9788E00A
:1033900012968C9312978285882321F0813009F050
:1033A000FEC515C084E79AE00E94CD2BF801838505
:1033B000882321F0843009F0F2C506C01092ED0890
:1033C00082E30E94D22AD4C50E94D00AD1C589E7DF
:1033D0009AE00E94CD2BD8011B968C911B978430CC
:1033E00009F0DDC50E942120C3C58EE79AE00E9446
:1033F000CD2BF8018681D70113968C931397978173
:1034000084818C5F8C7F292F2370822B14968C9360
:1034100014978091EE0816968C931697848183708A
:103420009C7F892B17968C931797808518968C9381
:10343000189719961C9219971A961C921A9787E05A
:103440001B968C931B971C961C921C978AE030CC81
:1034500088EA9AE068C584ED9AE00E94CD2BF801D5
:10346000248545858285882321F0813009F041C279
:1034700027C0C22EDD24942F80E0C82AD92A838554
:103480008130B1F0813020F0823009F087C112C064
:1034900080E061E0A6010E941B110E94B60A823002
:1034A00009F027C2CC2009F024C20E94BC0A21C224
:1034B00081E001C082E061E0A6010E941B1119C2F7
:1034C000F8018385813081F0813018F0823049F530
:1034D00016C0222319F02F3F29F402C080E015C046
:1034E00080E01AC080E01BC0222319F02F3F29F48E
:1034F00002C081E00AC081E00FC081E010C0222339
:1035000019F02F3F59F407C082E060E040E020E06E
:103510000E94DE1FEEC182E061E0F8CF82E062E04F
:10352000F7CFD8018681F701838317969C9117976F
:1035300014968C9114978C5F8C7F292F2370822B8B
:1035400084838091EE08868314968C9114978370FF
:103550009C7F892B878318968C91189780878CEC99
:1035600020C58EEF9AE00E94CD2B19820DC0F80184
:10357000E80FF11D83810E94462C8CE593E00E94A8
:10358000BB2B89818F5F89838981D80112969C9199
:103590001297891760F38EE493E00E94BB2BF80129
:1035A0008285882309F023C18385813009F44FC0C7
:1035B000813020F0823009F0E4C08FC080E0BE018D
:1035C000685F7F4F0E9406138985882319F0813038
:1035D00071F404C0F701148615860EC08FEFD70171
:1035E0001C968C931C971D961C921D9705C08A856E
:1035F000F70184878B85858781E0D7011E968C93A0
:103600001E979CE012969C9312979885913009F032
:10361000B5C082E01B968C931B978C85882319F08C
:10362000813071F404C0F7011786108A0EC08FEF45
:10363000D7011F968C931F9750961C92509705C0E8
:103640008D85F70187878E85808B81E08DC081E035
:10365000BE01685F7F4F0E9406138985882319F099
:10366000813071F408C0D7011C961C921C971D96DE
:103670001C921D970EC08FEFF7018487158609C035
:103680008A85D7011C968C931C978B851D968C93ED
:103690001D9782E0F70186879CE0928398859130A0
:1036A000C9F483878C85882319F0813049F403C0DD
:1036B0001786108A09C08FEFF7018787108A04C028
:1036C0008D8587878E85808B82E0F701818B8FE0E7
:1036D00082838DC081E083878AC082E0BE01685FFB
:1036E0007F4F0E9406138985882319F0813071F479
:1036F00004C0F701148615860EC08FEFD7011C9603
:103700008C931C971D961C921D9705C08A85F70106
:1037100084878B85858783E0D7011E968C931E97BF
:103720008CE012968C9312978885813031F582E077
:103730001B968C931B978C85882319F0813071F42C
:1037400004C0F7011786108A0EC08FEFD7011F96AD
:103750008C931F9750961C92509705C08D85F7014A
:1037600087878E85808B83E0D70151968C93519704
:103770008FE012968C9312973AC081E0F70183870D
:1037800036C088E29BE00E94CD2BD8011A968C911E
:103790000E94462C86E59BE00E94CD2BF801868195
:1037A000D70113968C931397978184818C5F8C7FBC
:1037B000292F2370822B14968C9314978091EE08F6
:1037C00016968C931697848183709C7F892B17960D
:1037D0008C931797808518968C9318978CEC199674
:1037E0008C9319971A961C921A9788E061CAF8016F
:1037F0008681D70113968C931397978184818C5F70
:103800008C7F292F2370822B14968C931497809190
:10381000EE0816968C931697848183709C7F892B73
:1038200017968C931797808518968C9318971996EE
:103830001C92199746C088E59BE00E94CD2BF801A9
:103840008285882319F08130A1F40CC0D7011B9622
:103850001C921B971C961C921C9719961C921997E8
:103860008AE00DC0F7018387148611868AE082837F
:1038700008C08CECD70119968C93199787E01296A3
:103880008C93F8018681D70113968C9313979781B7
:1038900084818C5F8C7F292F2370822B14968C93CC
:1038A00014978091EE0816968C93169784818370F6
:1038B0009C7F892B17968C931797808518968C93ED
:1038C00018971A961C921A9753C385E89BE02BC34E
:1038D0008FEA9BE00E94CD2BF8018685882319F0A2
:1038E0000E94C00A06C00E94B60A853011F40E94E8
:1038F000C80AD80116968C911697F70183831796FC
:103900009C91179714968C9114978C5F8C7F292F1C
:103910002370822B84838091EE08868314968C9189
:10392000149783709C7F892B878318968C911897A6
:103930008087118637C38AED9BE0F5C285E09CE065
:10394000F2C28DE29CE00E94CD2BD80116968C919C
:103950001697F701838317969C91179714968C916D
:1039600014978C5F8C7F292F2370822B8483809106
:10397000EE08868314968C91149783709C7F892B14
:10398000878318968C9118978087128688E08283A7
:103990001A968C911A978823A1F1813009F0E8C218
:1039A00019C188E59CE00E94CD2BD80116968C9118
:1039B0001697F701838317969C91179714968C910D
:1039C00014978C5F8C7F292F2370822B84838091A6
:1039D000EE08868314968C91149783709C7F892BB4
:1039E000878318968C9118978087128688E0828347
:1039F0001A968C911A97882321F0813009F0B8C269
:103A000002C08FEF14C1F8018385882319F00E944A
:103A100019207FC20E941D207CC280E89CE00E9489
:103A2000CD2B19820DC0F801E80FF11D83810E9492
:103A3000462C8CE593E00E94BB2B89818F5F8983A4
:103A40008981F8019281891770F38EE493E00E94D6
:103A5000BB2B6BC2D80118962C911897253009F40E
:103A60000AC1263060F42130B9F0213008F437C1A2
:103A7000223009F462C0233009F053C2AEC02730AF
:103A800009F4A3C1273008F46BC1283009F4DCC164
:103A9000293009F046C20EC28CE99CE00E94CD2B71
:103AA000F801C1849284D384A4848681D7011396BB
:103AB0008C931397978184818C5F8C7F292F23703F
:103AC000822B14968C9314978091EE0816968C9303
:103AD0001697848183709C7F892B17968C931797F8
:103AE000808518968C93189787E012968C93B0E196
:103AF000BA1510F482E813C20E941120882309F439
:103B000095C0CC2011F490E5C92E692D70E09D2D53
:103B100080E0682B792B9701265F3F4F8C2D4A2D33
:103B200050E00E943522882309F0A3C0D7011996DE
:103B30001C9219978A2D895FBBC881EC9CE00E947A
:103B4000CD2BF801C184A284D38444858681D7011A
:103B500013968C931397978184818C5F8C7F292F88
:103B60002370822B14968C9314978091EE081696EE
:103B70008C931697848183709C7F892B17968C93E6
:103B80001797808518968C93189787E012968C93D8
:103B90001297413110F082E84BC0488B0E941120EF
:103BA0004889882311F480E8BAC1CC2011F480E55B
:103BB000C82E6A2D70E09D2D80E0682B792B98012E
:103BC000235F3F4F8C2D50E00E94C524882311F0C5
:103BD00081E82DC0F7011186CBC187EE9CE00E94E1
:103BE000CD2BD80116968C911697F70183831796E3
:103BF0009C91179714968C9114978C5F8C7F292F2A
:103C00002370822B84838091EE08868314968C9196
:103C1000149783709C7F892B878318968C9180875B
:103C200087E082830E941120882331F480E8D70145
:103C300019968C9319979CC18CE7BE016F5F7F4FDB
:103C40000E949B208823A9F48981982F9161D80133
:103C500019962C911997222311F0816902C0892F9E
:103C60008F7789838CE769810E94C020882309F4BB
:103C700050C181E854C181E19DE00E94CD2BF80143
:103C80008681D70113968C931397978184818C5FDB
:103C90008C7F292F2370822B14968C9314978091FC
:103CA000EE0816968C931697848183709C7F892BDF
:103CB00017968C931797808518968C93189787E0A2
:103CC00012968C931297389A8FEF99E6A8E181505B
:103CD0009040A040E1F700C0000038981AC185E389
:103CE0009DE00E94CD2BF8018681D70113968C931D
:103CF0001397978184818C5F8C7F292F2370822B6F
:103D000014968C9314978091EE0816968C931697C0
:103D1000848183709C7F892B17968C93179780855D
:103D200018968C93189787E012968C931297199691
:103D30001C92199720E00FC0822F90E0F701E80F46
:103D4000F91F42E050E04C0F5D1F840F951FDC010E
:103D50008C9182872F5F253078F38CE0F70124C1A6
:103D600080E69DE00E94CD2BD80116968C91169787
:103D7000F701838317969C91179714968C9114974B
:103D80008C5F8C7F292F2370822B84838091EE0897
:103D9000868314968C91149783709C7F892B8783DC
:103DA00018968C911897808787E082838DEC8187A5
:103DB0008091EB03882309F4DBC0A701465F5F4FC6
:103DC0008CE061E00E94AE286AC08CE89DE0288B00
:103DD0000E94CD2BD80119968C9119978093430995
:103DE0001A968C911A978093440916968C9116977F
:103DF000F701838317969C91179714968C911497CB
:103E00008C5F8C7F392F3370832B84838091EE08F5
:103E1000868314968C91149783709C7F892B87835B
:103E200018968C9118978087288922838DEC81873A
:103E30008091EB03882309F49BC08CE061E043E4AC
:103E400059E00E948A2563C088EB9DE00E94CD2B3B
:103E5000D80116968C911697F701838317969C913B
:103E6000179714968C9114978C5F8C7F292F237051
:103E7000822B84838091EE08868314968C9114970C
:103E800083709C7F892B878318968C91808787E02D
:103E90008283B7016F5E7F4F88E40E9410298823D8
:103EA000E9F5D70112968C9112978E5F12968C933A
:103EB000129730C085EE9DE00E94CD2BD801199657
:103EC0006C9119976093430916968C911697F70198
:103ED000838317969C91179714968C9114978C5FF7
:103EE0008C7F292F2370822B84838091EE08868318
:103EF00014968C91149783709C7F892B87831896D6
:103F00008C91808787E0828388E40E94E928882357
:103F100029F4D70119961C9219972AC08FEFF7013F
:103F200026C080E19EE00E94CD2BD80116968C9190
:103F30001697F701838317969C91179714968C9187
:103F400014978C5F8C7F292F2370822B8483809120
:103F5000EE08868314968C91149783709C7F892B2E
:103F6000878318968C91808787E0828381EC818794
:103F7000D70111961C92119781E060960FB6F894C4
:103F8000DEBF0FBECDBFDF91CF911F910F91FF908C
:103F9000EF90DF90CF90BF90AF909F9008958CEC02
:103FA000F7018187128688E08283E2CF85EF98E06F
:103FB0000895FC018781869586950895982F842F12
:103FC000913099F0913018F0923051F51CC0609307
:103FD0003C093AE0632F0E94082F80934209822F08
:103FE0000E94082F80933E090895609341093AE0AA
:103FF000632F0E94082F80934709822F0E94082F69
:1040000080934009089560933B093AE0632F0E9432
:10401000082F80934609822F0E94082F8093580909
:1040200008958091B90308958091F2039091F3036C
:10403000089581E08093F103089581E08093F00377
:10404000089581E08093EF03089581E08093ED036C
:1040500008951F93CF93DF93CDB7DEB7C354D040FD
:104060000FB6F894DEBF0FBECDBF182F87E990E1E1
:104070000E94CD2B812F0E94462C8AE793E00E945C
:10408000BB2B809139098C8380E18D838091EE0870
:104090008F838091380988878C5F8093380982E00C
:1040A000898784E08A8782EF8B8787E08C878FE619
:1040B0008D871E878BE08B83CE0101960E941B1497
:1040C00081E08A83CE0101960E94DD101093B70330
:1040D000CD5BDF4F0FB6F894DEBF0FBECDBFDF91D3
:1040E000CF911F91089580913D09982F917080FD87
:1040F00008C08091FE03882321F01092FE0381E026
:1041000008959093FE0380E0089580913D09982FD3
:10411000917080FF08C08091FF03813021F081E021
:104120008093FF0308959093FF0380E0089590919A
:104130003D09892308950F931F93CF93DF930F9227
:10414000CDB7DEB78B0189830E94612989818160A7
:104150000E948429882321F40E94792981E00AC0E1
:1041600080E00E94BA2989830E9479298981F80117
:10417000808380E00F90DF91CF911F910F91089580
:104180001F93CF93DF9300D0CDB7DEB76A838983C7
:104190000E94612989810E9484296A81882321F4EF
:1041A0000E94792981E009C0862F0E948429182F56
:1041B0000E94792981E0111180E00F900F90DF912A
:1041C000CF911F9108951F93CF93DF930F92CDB797
:1041D000DEB780913C09813029F08130E0F08230F7
:1041E000F1F405C01092F6031092F70309C0809114
:1041F000F60390914209891728F48F5F8093F603A4
:1042000011E00EC08091F7038F5F8093F7039091C8
:104210003E09891721F41092F6031092F70310E07B
:1042200080914109813029F08130F0F0823001F530
:1042300006C01092F8031092F903126019C01260C0
:104240008091F80390914709891720F48F5F80933C
:10425000F8030EC01D7F8091F9038F5F8093F903EF
:1042600090914009891721F41092F8031092F903F4
:1042700080913B09813029F08130F0F0823001F5E6
:1042800006C01092FA031092FB03146019C0146068
:104290008091FA0390914609891720F48F5F8093EB
:1042A000FA030EC01B7F8091FB038F5F8093FB039B
:1042B00090915809891721F41092FA031092FB0388
:1042C0008091B903882311F18CE7BE016F5F7F4FA6
:1042D0000E949B208823D1F481E08093F40389819C
:1042E00080933D098F61898310FF02C08D7F898390
:1042F00011FF03C089818B7F898312FF03C08981ED
:10430000877F89838CE769810E94C0200F90DF91AD
:10431000CF911F9108951F93CF93DF9300D0CDB716
:10432000DEB7162F8CE7BE016F5F7F4F4A830E9476
:104330009B204A81882381F4642F61236161409529
:1043400089814823642B69838CE70E94C02091E017
:10435000882319F490E001C091E0892F0F900F900D
:10436000DF91CF911F9108951F93CF93DF930F9209
:10437000CDB7DEB789830E94612989810E94842993
:10438000882329F089E00E948429882321F40E944F
:10439000792981E009C080E00E948429182F0E94B9
:1043A000792981E0111180E00F90DF91CF911F9169
:1043B0000895CF92DF92EF92FF920F931F93CF93C6
:1043C000DF930F92CDB7DEB7F82E8B016A010E9402
:1043D00061298F2D0E948429882379F080E00E9432
:1043E0008429882351F00E946C29EE24E394EF285D
:1043F0008E2D0E948429882321F40E94792981E04E
:104400002AC080E00E94BA2989830E947929898183
:10441000F80180830E9461298F2D0E9484298823BE
:1044200061F081E00E948429882339F00E946C2980
:104430008E2D0E948429882321F40E94792982E00C
:104440000AC080E00E94BA2989830E947929898163
:10445000F601808380E00F90DF91CF911F910F9143
:10446000FF90EF90DF90CF900895AF92BF92CF92E0
:10447000DF92EF92FF920F931F93CF93DF930F92F0
:10448000CDB7DEB7182F062F6A01E22EA32E79834F
:104490000E946129812F880F0E94842979818823B5
:1044A00091F1872F0E948429882369F1802F0E942F
:1044B0008429882341F10E946C29812F880F816013
:1044C0000E9484298823F9F00E2D1A2DEE24FF2452
:1044D00056010894A108B1080FC0EA14FB0411F4B6
:1044E00080E001C081E00E94BA29F801808308942D
:1044F000E11CF11C0F5F1F4FEC14FD0471F70E94CB
:10450000792980E003C00E94792981E00F90DF9132
:10451000CF911F910F91FF90EF90DF90CF90BF90C0
:10452000AF900895EF92FF920F931F93CF93DF9375
:10453000CDB7DEB728970FB6F894DEBF0FBECDBF5C
:104540007C0180E560E070E048E050E09E012F5F74
:104550003F4F0E943522882309F044C0FE01319666
:1045600097E02191820F9150E1F781959885891705
:1045700031F08CE793E00E94BB2B82E034C00E81C7
:1045800010E083E0000F111F8A95E1F70115110576
:1045900039F180E5B80145E050E09E012F5F3F4FC3
:1045A0000E9435228823F1F42A819981920F8B8110
:1045B000980F3C81930F91953D81931731F082E9DB
:1045C00093E00E94BB2B84E00EC090E00596080F9C
:1045D000191F27FFDECFF7011183008380E003C09E
:1045E00083E001C081E028960FB6F894DEBF0FBECD
:1045F000CDBFDF91CF911F910F91FF90EF90089564
:104600009F92AF92BF92CF92DF92EF92FF920F9361
:104610001F93CF93DF93CDB7DEB7C850D1400FB60D
:10462000F894DEBF0FBECDBF6C01962E5A01FC017F
:10463000108280E560E070E048E050E09E012F5F6E
:104640003F4F0E943522882309F06DC0FE0131964C
:1046500097E02191820F9150E1F781959885891714
:1046600009F05BC00E8110E093E0000F111F9A95D6
:10467000E1F70115110509F452C080E5B80145E0E4
:1046800050E09E012F5F3F4F0E943522882309F0A2
:104690004AC08A819981890FEB808E0D9C81890F98
:1046A00081959D818917E9F5FF240B5F1F4F80E5F8
:1046B000B801A7019E01275F3F4F0E943522882342
:1046C00091F590E00AC049E050E04C0F5D1F240FC7
:1046D000351FF9012081920F8F5F282F30E02E15B2
:1046E0003F0588F391958C819817F9F4F601808144
:1046F0008F5F8083891559F4A114B10441F0F5014D
:10470000DE0119968DE00D9001928150E1F78A81CA
:1047100087FD0DC00E0D1F1DB0CF82E009C083E0E4
:1047200007C084E005C081E003C085E001C080E0EF
:10473000C85FDE4F0FB6F894DEBF0FBECDBFDF916E
:10474000CF911F910F91FF90EF90DF90CF90BF908E
:10475000AF909F9008957F928F929F92AF92BF9259
:10476000CF92DF92EF92FF920F931F93CF93DF933D
:10477000CDB7DEB7A1970FB6F894DEBF0FBECDBFA1
:1047800085E78B8384E48C8387E58D8383E48E8344
:104790001092EB0332E0E32EF12CEC0EFD1EC7016C
:1047A00060E040E050E00E94DC0A5E010894A11C39
:1047B000B11CC50160E040E050E00E9400238A8106
:1047C000882319F480E590E106C08981882309F0E7
:1047D0007DC089E690E10E94CD2B11E08CC0872D31
:1047E000982D6D2DAE014C5E5F4F0E94DC0A82E871
:1047F00090E10E94CD2B8E010C5E1F4F20E0F8014E
:1048000081918F0129A30E94462C8FEA93E00E9498
:10481000BB2B29A12F5F2D3091F78AE793E00E94EF
:10482000BB2B11E001E0AA24A3944AC0892D9C2D42
:10483000602FAE01495F5F4F0E9400238A8580335D
:1048400051F5112341F18DE890E10E94CD2B27E035
:10485000E22EF12CEC0EFD1E10E0F70181917F019C
:104860000E94462C8FEA93E00E94BB2B1F5F1D30F5
:10487000A1F78AE793E00E94BB2BCE014796BE01C9
:10488000665F7F4F4AE050E00E94442F009711F08E
:1048900011E001C010E08A85823389F48091EB0336
:1048A000882369F4CE010396BE01645F7F4F44E024
:1048B00050E00E94442F009711F4A092EB030F5F89
:1048C0008981801708F0B2CFD39407C011E0DD24AE
:1048D000D3947E2C8F2C9A2CCB2C8A818D1518F09A
:1048E000112309F07CCF91E0111190E08091EB034E
:1048F00089238093EB03812FA1960FB6F894DEBF36
:104900000FBECDBFDF91CF911F910F91FF90EF9020
:10491000DF90CF90BF90AF909F908F907F90089541
:104920000F931F93CF93DF9300D0CDB7DEB7062F41
:10493000142F7A8389830E9461298981880F0E94BC
:1049400084297A81882351F0872F0E948429882323
:1049500029F0802F0E948429882321F40E9479293C
:1049600081E00CC0812F0E9484290E9479298FE068
:1049700097E20197F1F700C0000080E00F900F90E0
:10498000DF91CF911F910F910895AF92BF92CF9277
:10499000DF92EF92FF921F93CF93DF93182F6B015B
:1049A0005A017901C0E0D0E00AC0F70141917F01CE
:1049B000BE016C0D7D1D812F0E9490242196CA1589
:1049C000DB0599F780E0DF91CF911F91FF90EF9089
:1049D000DF90CF90BF90AF900895AF92BF92CF92EB
:1049E000DF92EF92FF920F931F93CF93DF930F927B
:1049F000CDB7DEB7082F6A01E22EA32E69830E948D
:104A00006129802F880F0E94842969818823B9F049
:104A1000862F0E948429882391F00E946C29802F80
:104A2000880F81600E948429882349F00E2D1A2D59
:104A3000EE24FF2456010894A108B10813C00E9477
:104A4000792981E015C0EA14FB0411F480E001C06B
:104A500081E00E94BA29F80180830894E11CF11CCE
:104A60000F5F1F4FEC14FD0471F70E94792980E05D
:104A70000F90DF91CF911F910F91FF90EF90DF90FA
:104A8000CF90BF90AF900895CF92DF92EF92FF92B8
:104A90000F931F93CF93DF9300D0CDB7DEB77A018A
:104AA00069016A8389830E9461298981880F0E9434
:104AB00084296A81882381F0862F0E948429882393
:104AC00059F08601CC24DD240EC0F80181918F01BC
:104AD0000E948429882321F40E94792981E00FC053
:104AE0000894C11CD11CCE14DF0479F70E947929E7
:104AF0008FE097E20197F1F700C0000080E00F908F
:104B00000F90DF91CF911F910F91FF90EF90DF9069
:104B1000CF9008950F931F93CF93DF9300D0CDB71D
:104B2000DEB78A016A8389830E9461298981880F9F
:104B30000E9484296A818823E1F0862F83700E9475
:104B400084298823B1F0F80180810E948429882378
:104B500081F0F80181810E948429882351F00E940C
:104B600079298FE097E20197F1F700C0000080E01B
:104B700003C00E94792981E00F900F90DF91CF91BF
:104B80001F910F910895CF92DF92EF92FF92809143
:104B9000B9038093B8032091F5032093B903809162
:104BA000F403882389F030913D098091F2039091BC
:104BB000F30330FD03C08D7F816002C082608E7F71
:104BC0009093F3038093F203233009F470C12430EF
:104BD00048F48091B803213009F4AAC0223008F0CB
:104BE0002CC10DC0253009F4F0C1253008F469C18D
:104BF000263009F439C22B3009F063C26DC0882316
:104C0000A9F180E490E09093F3038093F20387B1DD
:104C10008F7687B9429A46988AE29EE00E94CD2B11
:104C200087E39EE00E94CD2B8091F3030E94462CE7
:104C30008091F2030E94462C8AE793E00E94BB2BEE
:104C40000E94FA291092FC0380E060E040E020E03E
:104C50000E94DE1F81E060E040E020E00E94DE1F55
:104C600082E060E040E020E00E94DE1F1092F4034A
:104C700035992EC00E94072B882329F08091FC03D0
:104C80008F5F8093FC038091FC03843608F419C283
:104C90004298863908F415C20E944B29882321F4D2
:104CA00082E49EE00E94CD2B1092FC038091F203DF
:104CB0009091F3038F7B80629093F3038093F203D0
:104CC00080E061E040E020E00E94DE1F8BE0F7C161
:104CD0001092FC03429AF5C18091E508882309F4FB
:104CE000F0C185E69EE00E94CD2BC090E303D090FA
:104CF000E403E090E503F090E6030E94AB23809389
:104D0000FD038091E3039091E4038C199D090E94B7
:104D1000FD2B80E89EE00E94CD2B0E94F62985E0C5
:104D20000E94292081E08093F5038093EC03C9C1A0
:104D3000813009F444C084E89EE00E94CD2B80912C
:104D4000B8038B3069F58091FD03882399F481E9DC
:104D50009EE00E94CD2B87E00E9429208091F203E3
:104D60009091F30380689093F3038093F20381E0C2
:104D700060E012C087EA9EE00E94CD2B88E00E948E
:104D800029208091F2039091F30391609093F303B3
:104D90008093F20381E061E040E020E00E94DE1FAA
:104DA00086EC9EE00E94CD2B8091F3030E94462C5E
:104DB0008091F2030E94462C81ED9EE07FC080919D
:104DC000F20387FF35C08091E508882389F180913F
:104DD000F403882361F00E947320882341F083ED5F
:104DE0009EE00E94CD2B80E00E94292015C080917A
:104DF000F4038823A1F08091EC03882381F0809153
:104E00003D0980FD0CC08DEE9EE00E94CD2B80E020
:104E10000E9429201092EC0382E08093F503809198
:104E2000F103882329F084E08093F5031092F103C5
:104E3000359B47C18BE09FE039C18230A1F080E211
:104E40009FE00E94CD2B8DE29FE00E94CD2B8091B0
:104E5000F3030E94462C8091F2030E94462C8AE7BD
:104E600093E00E94BB2B0E948520882351F088E3A9
:104E70009FE00E94CD2B81E00E94292081E0809359
:104E8000F503359B09C08CE49FE00E94CD2B86E0A2
:104E90000E9429201092F5038091F103882309F4E0
:104EA00010C184E08093F5031092F1030AC1809150
:104EB000B803833009F405C181E69FE00E94CD2B41
:104EC00000C18091B803843071F18091F203909118
:104ED000F3038B7F9093F3038093F2038EE69FE0BE
:104EE0000E94CD2B8BE79FE00E94CD2B8091F30396
:104EF0000E94462C8091F2030E94462C8AE793E0A0
:104F00000E94BB2B469A1092FC038091EB038823EE
:104F100051F08CE061E045EB53E00E948A2586E881
:104F20009FE00E94CD2B0E94072B882339F08091AF
:104F3000FC038F3118F48F5F8093FC038091FC0396
:104F40008E3159F48CE760E040E40E948B2182E0CE
:104F500061E040E020E00E94DE1F0E94852088235F
:104F6000A1F08091F2039091F30382608E7F909381
:104F7000F3038093F20381EA9FE00E94CD2B81E04E
:104F80000E94292085E08093F5038091EF03882318
:104F900019F085E08093F503359B93C085EB9FE086
:104FA0000E94CD2B86E00E9429208091EB0388236C
:104FB00009F481C08CE061E041EB53E00E948A2556
:104FC0008AEC9FE00E94CD2B76C08091B80385309B
:104FD00041F180EE9FE00E94CD2B8DEE9FE00E947C
:104FE000CD2B8091F3030E94462C8091F2030E9406
:104FF000462C8AE793E00E94BB2B82E060E040E011
:1050000020E00E94DE1F8091EB03882351F08CE0AA
:1050100061E041EB53E00E948A2588EF9FE00E9407
:10502000CD2B8091EF03882389F08091F20390913A
:10503000F30384609093F3038093F20387B18F7638
:1050400087B982E00E9429201092EF038091F0033B
:10505000882329F086E08093F5031092F003359BB6
:1050600030C08EE090E122C08091B8038630D1F04C
:105070008CE760E440E40E948B21469883E290E153
:105080000E94CD2B80E390E10E94CD2B8091F30311
:105090000E94462C8091F2030E94462C8AE793E0FE
:1050A0000E94BB2B359B0AC08BE390E10E94CD2B65
:1050B00086E00E9429201092F50303C081E08093CE
:1050C000F5038091ED03882309F443C08091F20336
:1050D00080FF03C080E00E9429208091F20381FFBD
:1050E00003C081E00E9429208091F20382FF03C067
:1050F00082E00E9429208091F20383FF03C083E0B5
:105100000E9429208091F20384FF03C084E00E9462
:1051100029208091F20385FF03C085E00E942920A9
:105120008091F20386FF03C086E00E9429208091CF
:10513000F20387FF03C087E00E9429208091F203D9
:105140009091F30390FF03C088E00E942920109201
:10515000ED03FF90EF90DF90CF900895EF92FF92D4
:105160001F93CF93DF930F92CDB7DEB7182F7A013D
:1051700069830E946129812F880F0E948429698197
:105180008823E9F0862F83700E9484298823B9F050
:105190000E946C29812F880F81600E9484298823B6
:1051A00071F081E00E94BA29F701808380E00E94BB
:1051B000BA29F70181830E94792980E003C00E9407
:1051C000792981E00F90DF91CF911F91FF90EF90AF
:1051D0000895CF93DF9300D0CDB7DEB76A8389837C
:1051E0000E9461298981880F0E9484296A8188230D
:1051F00029F0862F0E948429882321F40E9479298E
:1052000081E009C00E9479298FE097E20197F1F7C8
:1052100000C0000080E00F900F90DF91CF910895C3
:10522000CF92DF92EF92FF920F931F93CF93DF9372
:105230000F92CDB7DEB77B0189830E9461298981F6
:10524000880F81600E948429882321F40E94792993
:105250008FEF17C081E00E94BA29182F00E080E08C
:105260000E94BA29C82EDD24C02AD12A0E94792999
:10527000E114F10411F48D2D04C0F701D182C08234
:1052800080E00F90DF91CF911F910F91FF90EF90F1
:10529000DF90CF9008958BB18F7C8BB98AB18F7CD2
:1052A0008AB989E096E09A95F1F700C0549A96E0A1
:1052B0009A95F1F700C054988150A1F789B1807296
:1052C0000895559A86E08A95F1F700C0549A86E0D1
:1052D0008A95F1F700C00895559886E08A95F1F710
:1052E00000C0549886E08A95F1F700C00E946129B9
:1052F0000895549886E08A95F1F700C0559886E0A5
:105300008A95F1F700C00895F89428E030E090E81D
:10531000492F482311F4559A01C0559846E04A9503
:10532000F1F700C054984DE04A95F1F70000549A07
:1053300046E04A95F1F700C096952150304041F77C
:10534000559886E08A95F1F700C0549846E04A9552
:10535000F1F700C099B186E08A95F1F700C0549A40
:10536000559A46E04A95F1F700C0789481E095FDA2
:1053700080E00895282FF894559898E080E0880FF1
:1053800036E03A95F1F700C0549836E03A95F1F7D7
:1053900000C04D99816036E03A95F1F700C0549A0B
:1053A00036E03A95F1F700C0915049F7222311F009
:1053B000559A01C0559896E09A95F1F700C0549817
:1053C0003DE03A95F1F70000549A559A96E09A9587
:1053D000F1F700C07894089580910004882319F0B3
:1053E0008BE090E0089589E090E0089581E080935B
:1053F000000408951092000408958BB18F738BB947
:105400008AB18F738AB90895579A86E08A95F1F721
:1054100000C0569A86E08A95F1F700C00895579823
:1054200086E08A95F1F700C0569886E08A95F1F7F4
:1054300000C00E94042A0895569886E08A95F1F7E4
:1054400000C0579886E08A95F1F700C0089528E0DB
:1054500030E090E8492F482311F4579A01C057983B
:1054600046E04A95F1F700C056984DE04A95F1F7AD
:105470000000569A46E04A95F1F700C096952150F3
:10548000304041F7579886E08A95F1F700C056986A
:1054900096E09A95F1F700C089B146E04A95F1F798
:1054A00000C0569A579A96E09A95F1F700C08095F9
:1054B000881F8827881F0895282F579898E080E034
:1054C000880F36E03A95F1F700C0569836E03A95E5
:1054D000F1F700C04F99816036E03A95F1F700C0CE
:1054E000569A36E03A95F1F700C0915049F72223D9
:1054F00011F0579A01C0579896E09A95F1F700C0BD
:1055000056983DE03A95F1F70000569A579A96E082
:105510009A95F1F700C0089590915B0983B1809549
:1055200089279091010498239095909301042091EC
:105530000204282329272093020498239223809190
:105540005B09892780935B0920915A0980915B0947
:105550008923822B80935A092091590980915B09F4
:1055600080958923822B809359090895F89490910E
:105570005A09892390915A09982790935A09789447
:105580000895F89490915909892390915909982781
:105590009093590978940895F89490915B097894C0
:1055A000892308958093070481E080930604089579
:1055B00010920604089581E090910604992309F45D
:1055C00080E0089580910704882329F0815080931A
:1055D000070480E0089581E008958093050481E048
:1055E00080930404089510920404089581E090913A
:1055F0000404992309F480E0089581E09091050462
:10560000911180E0089581E08093030408958091D2
:105610000304882321F01092030481E0089580E0C0
:1056200008951092C5008CE08093C40088E98093AF
:10563000C1001092DE091092DC091092DD0910926F
:105640005F0A08959091DC092091DE0991509F77BF
:105650002917C1F3E091DE09F0E0E152F64F8083B3
:105660008091DE098F5F8093DE098091DE098038AA
:1056700011F41092DE098091C10080628093C10014
:1056800008953091DD0920915F0A3217A1F0209131
:105690005F0AE22FF0E0E45AF64F3081FC013083DC
:1056A0002F5F20935F0A80915F0A803831F4109257
:1056B0005F0A80E0089581E0089580E008951F92D8
:1056C0000F920FB60F920BB60F9211248F939F93E8
:1056D000EF93FF93E091DC09F0E0E152F64F808117
:1056E0008093C6008091DC098F5F8093DC098091F4
:1056F000DC09803811F41092DC099091DE09809168
:10570000DC09981729F48091C1008F7D8093C10036
:10571000FF91EF919F918F910F900BBE0F900FBE55
:105720000F901F9018951F920F920FB60F920BB605
:105730000F9211248F939F93EF93FF938091DD0934
:10574000E82FF0E09091C600E45AF64F90838F5F07
:105750008093DD098091DD09803811F41092DD0914
:10576000FF91EF919F918F910F900BBE0F900FBE05
:105770000F901F901895CF93DF93EC0108C08A30EB
:1057800019F48DE00E94222B89910E94222B88819E
:105790008823A9F7DF91CF9108951F93CF93DF93CB
:1057A000EC012196FC0114911A3019F48DE00E944D
:1057B000222B812F0E94222BFE012196149111236E
:1057C00099F7DF91CF911F9108950F931F93CF9376
:1057D000DF93082FC8E0D0E010E8812F802311F07C
:1057E00081E301C080E30E94222B16952197A9F73F
:1057F000DF91CF911F910F910895DF92EF92FF9269
:105800000F931F93CF93DF93CDB7DEB729970FB6D2
:10581000F894DEBF0FBECDBF8C01DE011196EAEB1E
:10582000F3E088E001900D928150E1F77E01089449
:10583000E11CF11C84E0D82E91E010C08F5F021BA8
:10584000130B90E002171307C8F7992329F4805D22
:1058500099870E94222B9985DA9431F0F7012191E2
:1058600031917F0180E0EECF802F805D0E94222B5E
:1058700029960FB6F894DEBF0FBECDBFDF91CF9152
:105880001F910F91FF90EF90DF9008951F93CF939A
:10589000DF93CDB7DEB760970FB6F894DEBF0FBECB
:1058A000CDBF182FDE011196E2ECF3E080E101900C
:1058B0000D928150E1F7812F82958F70E1E0F0E049
:1058C000EC0FFD1FE80FF11D80810E94222B1F703D
:1058D000E1E0F0E0EC0FFD1FE10FF11D80810E947F
:1058E000222B60960FB6F894DEBF0FBECDBFDF91BE
:1058F000CF911F910895CF93DF93CDB7DEB7C354F7
:10590000D0400FB6F894DEBF0FBECDBF1092E508B1
:1059100080E880BFA89528E288E190E00FB6F8946F
:10592000A895809360000FBE209360001092E90854
:105930001092EA081092EB081092EC081092EF080F
:105940000E94112B0E9476080E94FD290E94D61FFA
:105950009093F4088093F30889E0809381008FE3AB
:105960009FE1909389008093880082E080936F008C
:105970002C9885B1806685B984B1806784B94098D8
:10598000389A139A149881B1886181B915980D9A43
:1059900046983E9A5A9852985B98539A429A3A9AE5
:1059A00088B18F7688B987B18F7687B980E060E15A
:1059B00041E254E029E234E00E94011181E060E21A
:1059C00041E154E029E334E00E94011182E060E407
:1059D00049E154E021E334E00E9401111092ED0806
:1059E000789481EE93E00E94CD2B1092E8088DE12F
:1059F00093E00E94BB2B0E94B60E0E94FD2B8AEF03
:105A000093E00E94CD2B8CEF93E00E94CD2B8091F0
:105A100060000E94462C85E094E00E94CD2B87E038
:105A200094E00E94CD2B84E393E00E94BB2B80E1A5
:105A300094E00E94CD2B86E294E00E94CD2B8CE274
:105A400094E00E94CD2B8CE394E00E94CD2B82E465
:105A500094E00E94CD2B8DE494E00E94CD2B86E54E
:105A600094E00E94CD2B8BE594E00E94CD2B87E63D
:105A700094E00E94CD2B8BE694E00E94CD2B84E72E
:105A800094E00E94CD2B86E794E00E94CD2B84B752
:105A90000E94462C8EE794E00E94CD2B14BE0E94FB
:105AA000D3138093EE080E94590F8AE393E00E947B
:105AB000BB2B8091EE080E94462C8BE493E00E9461
:105AC000BB2B0E94210E80E28093390910923A0983
:105AD00000E010E0FF24FA94A8950E945A0E0E945C
:105AE0003E098091E3088823B1F080E960EE78E018
:105AF0000E942E1382E966EE78E00E942E130E9427
:105B0000EC298A30910528F088E461EF78E00E9462
:105B100010291092E3080E94C3258091E40888238D
:105B200021F00E94E3201092E4080E94690F88236C
:105B300011F0A895FACF0E94D90F8091F3089091A7
:105B4000F408FC01208120FF2AC00E944814E09143
:105B5000F308F091F40890819E7F90838823F9F4F4
:105B6000CF010E9415142091F3083091F408882386
:105B700089F4C901BE016F5F7F4F0E946F148823B3
:105B800071F0CE0101960E941B14CE0101960E9475
:105B9000DD1005C0C9010E94D91F0E94FB10809131
:105BA000F008882309F498CF0E94DB2A882379F033
:105BB0000E94E22A882359F081E08093ED080E9438
:105BC000D82A80E894E00E94CD2B00E010E080917C
:105BD000E9089091EA08A091EB08B091EC080196D1
:105BE000A11DB11D8093E9089093EA08A093EB08EA
:105BF000B093EC0880E00E94B81181E00E94B811D7
:105C000082E00E94B8118091ED08843009F454C0FC
:105C1000853040F48130B9F0813070F0833009F084
:105C20008EC031C0863009F47CC0863008F461C073
:105C3000873009F084C077C00D9A389A139A149867
:105C40001092EF087CC080E00E94EA08F2E08C3BF2
:105C50009F0708F474C00F5F1F4F0230110509F051
:105C60006EC083E08093ED081398149A8AE994E05B
:105C70000E94CD2B8091E9089091EA080E94FD2BAB
:105C800083EC94E016C00F5F1F4F0531110508F437
:105C900056C0389884E08093ED0886EC94E00E942A
:105CA000CD2B8091E9089091EA080E94FD2B86EFA8
:105CB00094E00E94CD2B41C0319B41C081E0809394
:105CC000E5080F5F1F4F06301105C8F10D9885E0FC
:105CD0008093ED0889EF94E00E94CD2B8091E90834
:105CE0009091EA080E94FD2B87E295E00E94CD2B5F
:105CF00026C08091EF08882311F58AE295E00E9482
:105D0000CD2B8091E9089091EA080E94FD2B8DE34C
:105D100095E00E94CD2B0E94EC0E81E08093EF086D
:105D20000EC00D9A0CC0389A139A149881E0809393
:105D3000E8081092ED081092EF0800E010E0E09003
:105D4000ED08FE1409F441C022E0E216B9F02E1568
:105D500030F081E0EE2071F0E816B9F50AC0E5E018
:105D6000EE16E1F0F7E0EF1621F124E0E21669F516
:105D70000AC081E060E041E050E01FC081E060E0E7
:105D800042E050E01AC081E060E040E050E00E9454
:105D90001B1182E060E042E050E015C081E060E06D
:105DA00040E050E00E941B1182E060E041E050E0E2
:105DB0000AC081E060E040E050E00E941B1182E0F8
:105DC00060E040E050E00E941B111092F008FE2CB1
:105DD00083CE629FD001739FF001829FE00DF11D81
:105DE000649FE00DF11D929FF00D839FF00D749F55
:105DF000F00D659FF00D9927729FB00DE11DF91F01
:105E0000639FB00DE11DF91FBD01CF01112408955D
:105E1000991B79E004C0991F961708F0961B881FFC
:105E20007A95C9F78095089597FB092E07260AD021
:105E300077FD04D00CD006D000201AF4709561953F
:105E40007F4F0895F6F7909581959F4F0895AA1B6F
:105E5000BB1B51E107C0AA1FBB1FA617B70710F055
:105E6000A61BB70B881F991F5A95A9F78095909587
:105E7000BC01CD010895FB01DC0102C005900D922B
:105E800041505040D8F70895FB01DC0104C08D91CA
:105E90000190801921F441505040C8F7881B990B9C
:105EA0000895FB01DC0102C001900D924150504069
:105EB000D8F70895DC01CB01FC01F999FECF06C0AB
:105EC000F2BDE1BDF89A319600B40D9241505040B8
:105ED000B8F70895F999FECF92BD81BDF89A992738
:105EE00080B50895DC01CB0103C02D910E947D2F68
:105EF00041505040D0F70895262FF999FECF1FBA90
:105F000092BD81BD20BD0FB6F894FA9AF99A0FBEE2
:085F100001960895F894FFCFFB
:105F18000A0001FFFF204552524F5221003A20301B
:105F280078000A002E2E2E204552524F52210A0088
:105F38002E2E2E20646F6E65210A00646F6E652117
:105F48000A00205265616420556E697175652D4996
:105F5800443A200020525F4552524F522100206D92
:105F6800560A0020000A0A383330304C3E0A0075C1
:105F78006E6B6E6F776E20636F6D6D616E640A0075
:105F8800383330304C3E00535441540048454C504F
:105F98000052544D310052544D320052544D33008A
:105FA80052544D340052544D350052544D3600521F
:105FB800544D370052544D3800564F4C54005052EF
:105FC8004F4D004944004441435700444143520067
:105FD800007702D50D7C02E90B8102AE0D8602879F
:105FE8000D8B02750D90026C0D9502630D9A025A85
:105FF8000D9F02E30BA4021B0DA902C50CAE02699A
:106008000CB302830CB6021A0CBB02EF0BC00200E1
:10601800000A00726571206F75742064726F707069
:10602800656420616674657220330A000A4D6F64E6
:10603800756C652053657269616C204E756D62657B
:10604800723A2000322E372E33004D6F64756C651E
:1060580020416464726573733A20000A0A000A00DA
:106068006F6666733A0020636E743A002000322E21
:10607800372E330036061B068E07DB054E070E0744
:10608800CE069B055B058E064E060A0072746D20CF
:10609800636D6E206864722063686B206661696C4A
:1060A8000A006D756C7420686561646572206368A8
:1060B80065636B73756D206572726F72210A0020BB
:1060C8000020002FFC2C1C06FFFF1027E8036400AB
:1060D8000A00303132333435363738394142434497
:0260E80045462B
:00000001FF
